:0600000083018B018A015F
:06000600850186018C015A
:06000C009D018F0190012F
:060012009101920193012F
:060018009401950198011E
:06001E0099019A01AB01FB
:06002400AC01AA018316E5
:06002A0010308500FF30DC
:0600300086008117640048
:06003600A73081008312D7
:06003C008501860105119B
:06004200051085101530C9
:060048009E009F019F0BCA
:06004E0026289E0B262867
:060054000F30860530307C
:06005A00860483160F303E
:0600600006058600831274
:060066000515051107302D
:06006C009E009F019F0BA6
:0600720038289E0B38281F
:0600780005150511013021
:06007E009E009F019F0B94
:0600840041289E0B4128FB
:06008A000F308605203056
:06009000860405150511B0
:060096002830F8200830BC
:06009C00F8200130F820FD
:0600A2000C30F8200630CE
:0600A800F8200730A10062
:0600AE001321A40008303C
:0600B400A1001321A500CC
:0600BA000B30A100132130
:0600C00003192A150F30A0
:0600C600A1001321031943
:0600CC008D284530E520FF
:0600D2004530E5202D3051
:0600D800E5204930E5209F
:0600DE004E30E520493020
:0600E400E5205430E52088
:0600EA003A30E5200B2175
:0600F0000030A100210810
:0600F6008900B62088001D
:0600FC001C214030803899
:06010200F820C7202108CF
:06010800A520E5200B21FB
:06010E0021080F3C031C58
:060114008D28A10A7A28E3
:06011A000130F820061C74
:06012000522A6E2982073D
:06012600003400340A342D
:06012C00003400346434CD
:0601320000340334E83440
:06013800003427341034EE
:06013E0001348634A034F8
:060144000F344234403488
:06014A008207303431345D
:0601500032343334343474
:0601560035343634373465
:06015C003834393441344F
:0601620042344334443432
:0601680045344634820715
:06016E000D34BC343634F0
:060174000D34BB340A3417
:06017A00003414340134CE
:0601800000340034FF34DE
:06018600FF3428340A34A6
:06018C0000348316F03080
:060192000604860018308F
:0601980085008312051032
:06019E008514051506089A
:0601A400F0399B0005117B
:0601AA0000000000051535
:0601B0000511060E0F39D7
:0601B6001B049B1BC7287F
:0601BC00851083160F30D0
:0601C20006058600831211
:0601C80008009600C720AC
:0601CE000F308605160843
:0601D400F03986048510DD
:0601DA00051405150511D6
:0601E0000F308605160E2B
:0601E600F0398604051546
:0601EC0005110800960059
:0601F200C7200F30860556
:0601F8001608F039860430
:0601FE0085100510051537
:0602040005110F30860514
:06020A00160EF039860417
:06021000051505110800B0
:06021600FF309E009F0175
:06021C009F0B0E299E0B52
:060222000E290800831202
:0602280021088900831685
:06022E0008148312080809
:06023400A2000800831681
:06023A008B13081555307E
:060240008900AA308900CC
:0602460088148818242929
:06024C008B1708002A12C6
:060252000F0893020318DF
:0602580033299403940A0F
:06025E00031D3229950387
:060264009403100894024F
:06026A000318382995037A
:06027000110895020318BD
:060276002A1608002A12FE
:06027C000F089307031CAC
:060282004829940F4829F1
:0602880001309507031888
:06028E002A161008940777
:06029400031C4D29950A30
:06029A001108950703188E
:0602A0002A1608002708E1
:0602A6008F002808900003
:0602AC0029089100080082
:0602B2002A1301301302C3
:0602B80003186329013068
:0602BE001402031863297D
:0602C4002A170800A1004A
:0602CA0013219500A10ABA
:0602D00013219400A10AB5
:0602D60013219300080053
:0602DC0000308038F8201C
:0602E200C7204530E520B5
:0602E8004530E520503016
:0602EE00E5205230E5207E
:0602F4004F30E5204D3003
:0602FA00E5202030E520A4
:0603000040308038F820B7
:06030600C7204D30E52088
:06030C004F30E5204430F3
:06031200E5204530E52066
:060318002030E520313029
:06031E00E5202E30E52071
:060324003330E5200B213F
:06032A000B210B21060867
:060330000F39031D6E29C8
:060336000130F820C72091
:06033C00A101A201A301D2
:06034200061CAA29A10A15
:0603480021080F3C031C1C
:06034E00A1010B212310A8
:06035400861CAE29A20A7E
:06035A000B21061DB22973
:06036000A2030B21861D23
:06036600D3290B21210840
:06036C0089002208880050
:060372001C210130F820FF
:06037800C7202A30E52039
:06037E005330E520413080
:06038400E5205630E520E3
:06038A004530E52044307F
:06039000E5202A30E52003
:060396000B210B210B21DD
:06039C000B210130F820E6
:0603A200C720A301413059
:0603A800E5204430E520D1
:0603AE004430E52052304E
:0603B400E5203A30E520CF
:0603BA002318E1291321C4
:0603C00023142108F039AE
:0603C6008E000E0EA520C2
:0603CC00E52021080F39B5
:0603D200A520E5204030EB
:0603D8008038F820C72068
:0603DE004430E52041302F
:0603E400E5205430E52085
:0603EA004130E5203A302D
:0603F000E5202208F039AF
:0603F6008E000E0EA52092
:0603FC00E52022080F3984
:06040200A520E5200030FA
:060408008038F820C72037
:06040E00A1299B010C086E
:060414009C0092209802FA
:06041A000318182A01304E
:0604200099020318182ADE
:0604260001309A020318E8
:06042C00182A1B149C03BA
:060432001C089220990253
:060438000318232A013025
:06043E009A020318232AB4
:060444001B149C031C08C0
:06044A0092209A02031843
:060450002B2A03142C2AE4
:060456001B0C00349B01A9
:06045C000C089C00922038
:060462009807031C3D2A6F
:0604680001309907031C9E
:06046E003D2A01309A074F
:06047400031C3D2A1B14CD
:06047A009C031C08922007
:060480009907031C482A45
:0604860001309A07031C7F
:06048C00482A1B149C032A
:060492001C0892209A07ED
:06049800031C502A0314AE
:06049E00512A1B0C003482
:0604A40011308C0009304C
:0604AA008D008E010630FA
:0604B0009D000822031864
:0604B600632A8E0A8D038B
:0604BC00031D592A033064
:0604C2008C02662A2D22C7
:0604C80003308C02093034
:0604CE008D0010301D0737
:0604D4009B009B031B08C6
:0604DA0084000E088E01F3
:0604E00080009D030130C5
:0604E6000C07031D592A5A
:0604EC0018088F00AA1E93
:0604F2007C2A06108611B1
:0604F80006309D00210802
:0604FE000605A200A21990
:060504008F2A0730803849
:06050A00F820C72020309C
:06051000E5200B308038ED
:06051600F820C720203090
:06051C00E52000308038EC
:06052200F820C720860846
:06052800A1000F301D07C9
:06052E008400000803191F
:060534009E2A3038E5208C
:06053A00A72A06301D0295
:06054000031DA52A203076
:06054600E520A72A303079
:06054C00E5202A1DB02A83
:060552000C30A100132192
:06055800031DB22AAA17E0
:06055E00B62A8619B62A38
:06056400AA130230A600FC
:06056A00BD2A0130A600CD
:060570000A30A100132176
:06057600031DC32A260844
:06057C001D02031DC32A4D
:060582002E30E5202A1DC9
:06058800C82AAA1BCC2AC0
:06058E00CA2A8619CC2ADE
:060594000530CD2A043001
:06059A001D02031DD22A20
:0605A0002E30E5200930B9
:0605A600A1001321031D5A
:0605AC00DF2A01301D02F0
:0605B200031DDF2A4030AA
:0605B8008038F820C72086
:0605BE009D0B952A0A3096
:0605C400A1001321031D3C
:0605CA00EC2A0F301D07B2
:0605D00084000008303831
:0605D600E5202030E520C5
:0605DC004D30E52048301F
:0605E200E5207A30E5205F
:0605E8002A1DFF2A20304D
:0605EE00E5202A1CFD2A95
:0605F4004C30E520FF2A57
:0605FA002030E520003076
:060600008038F82097018C
:060606008101000000006C
:06060C009D01C7309E00B5
:060612000B309F000530D3
:06061800A0008B01103070
:06061E00850083161F3069
:06062400850083120B1D8E
:06062A00192B970A0B11C9
:060630001C2B000000007D
:0606360000009E0B142BD6
:06063C00C7309E009F0B79
:06064200142B0B309F0099
:06064800A00B142B0610AC
:06064E00861182308E00CF
:060654000B1D2F2B970A7D
:06065A000B11322B000021
:06066000000000008E0BFB
:060666002A2B24088E007F
:06066C008E0B362B250861
:060672008E0000008E0B5B
:060678003A2B030186008D
:06067E0010308500831618
:060684001730850083120F
:06068A000B19970A0B1189
:06069000010899001708A3
:060696009A009B019B0A83
:06069C00851585110B110C
:0606A20001081902031912
:0606A8004D2B9B0A9B098B
:0606AE009B0A1B0A9800E4
:0606B400103085008316E2
:0606BA00043085008312EC
:0606C0002A1DDF2B1808C3
:0606C600930019089400E6
:0606CC001A0895008316D8
:0606D200F630060586006B
:0606D80083122A18A62B74
:0606DE000D30A100132104
:0606E4002B02031D782B20
:0606EA00AA18812B7A2BF7
:0606F000AB0ADF2B180825
:0606F600A7001908A8008E
:0606FC001A08A900AA146F
:06070200522128215921BB
:060708002A1F902B0E30A9
:06070E00A10013212C02E2
:06071400031DDE2B2A1478
:06071A00AA10AC01DF2B68
:0607200005308F0090017E
:0607260091012A1EA02B28
:06072C00FA308F00FF30DF
:060732009000FF30910071
:060738003D212A1AA32B4B
:06073E00862B3D212A1A62
:06074400862BAB01AA1098
:06074A00DF2BAA12522170
:06075000282159212A1B9B
:06075600DC2B13089B00E0
:06075C002A1ACB2B061443
:0607620086119B0A031939
:06076800B72B9B0A0319E8
:06076E00AA1691019001A2
:060774000A308F003D2158
:06077A002A1ADC2B0E30F0
:06078000A10013212C0270
:060786000319C72BAC0AA9
:06078C00DF2B2A10AC0176
:06079200AB01DF2B061095
:0607980086159B03031906
:06079E00D22B9B0303199E
:0607A400AA16F6308F00DA
:0607AA00FF309000FF305B
:0607B00091003D212A1A10
:0607B600BF2BAC01DF2B9C
:0607BC00AC0A8618E42BD4
:0607C20000306421E62B6B
:0607C8000330642106303D
:0607CE00A1001321031934
:0607D400FE2B0619FE2BAE
:0607DA001A089100190845
:0607E000900018088F00D4
:0607E6000519F72B282184
:0607EC00F82B3D21150869
:0607F2009A0014089900B2
:0607F80013089800522ACC
:0207FE00FF3FBB
:084000000F000F000F000F007C
:02400E00F93F78
:00000001FF
